:1000000018C130C12FC12EC12DC12CC12BC162C35B
:1000100029C128C127C141545A0D00415445300D12
:100020000041542B435042533D22534D220D004179
:10003000542B435042523D310D00415445310D0087
:1000400041542B434D47533D35360D00303031314F
:100050003030304239310030303038414132413077
:100060003432323034323030343135303431323071
:100070003431453034313330343130303032313056
:100080003032303034323330343334303433303053
:100090003434303034334430343442303433393013
:1000A0003032303034333430343330303434323032
:1000B0003032451A0D003030303841413241303451
:1000C0003232303432303034313530343132303411
:1000D00031453034313330343130303032313034F6
:1000E00031453034343230343341303434303030D0
:1000F00032453034313130343330303433333034CE
:1001000033303034333630343344303433383034B1
:1001100033411A0D003030303841413241303432F1
:1001200032303432303034313530343132303431B1
:100130004530343133303431303030323130303298
:10014000303034314530343432303433413034346B
:100150003030303245303032303034333430343374
:100160003230343335303434303034333830303268
:10017000451A0D003030303841413241303432328E
:10018000303432303034313530343132303431453E
:10019000303431333034313030303231303032304D
:1001A000303431453034343230343341303434300B
:1001B0003030324530303230303433413034333007
:1001C00030343346303433453034343230303245D5
:1001D0001A0D003030303841413241303431323044
:1001E00034334430343338303433433034333030C4
:1001F00034334430343338303433353030323130C6
:1002000030323030343144303433353034343230BD
:1002100030323030343346303433383034343230A6
:100220003433303034334430343338303434461A95
:100230000D0011241FBECFEDCDBF10E0A0E6B0E051
:10024000E8EEF7E003C0C89531960D92A837B107E4
:10025000D1F710E0A8E7B0E001C01D92A939B107BD
:10026000E1F701C0CDCECEEDD0E0DEBFCDBF0ED1E7
:1002700081E061D18AEF0FD260E070E086E190E02A
:100280000FD1882339F017E08AEF05D21150E0F73B
:1002900082E0EFCF60E070E08BE190E001D1882355
:1002A00011F082E048D160E070E081E290E0F8D0A7
:1002B000882311F083E03FD15DD28FE290E035D208
:1002C0008AEFE9D18AEFE7D119828C2F9D2F019611
:1002D00049D2082F192F89818C30C8F584E0C9CF05
:1002E00084E029D10F2EF0EFFF2EF02D49C081E8D8
:1002F00022D146C083818093600082818093610017
:1003000085818093620084818093630087818093DC
:100310006400868180936500818580936600808576
:10032000809367008385809368008285809369004D
:1003300086E480936A00848580936B0010926C0041
:1003400082E8F9D00F2EF1EFFF2EF02D3DC0FF24F3
:10035000F12FE02F8081882399F0F12FE02FEF0D0E
:10036000F11D80818F3409F4BBCF823409F4BFCFF3
:10037000F394F12FE02FEF0DF11D8081882369F7B1
:10038000F0E8FF1508F476CF8F2D9927282F392F05
:10039000F12FE02FE80FF91F80818823A9F0F12FBA
:1003A000E02FE20FF31F8081823221F481818B32B2
:1003B00009F4A0CFF3942F2D3327F12FE02FE20F74
:1003C000F31F8081882359F78BED8F1510F085E09E
:1003D00050CFDD24D394CC24869B0CC0E4E6ED15ED
:1003E00018F4C798DD24D39484E655D1C79AD394E2
:1003F0008699F4CF82E34FD18699EECFDD2019F0B4
:100400008AE058D1DD24C394C3FE02C0C79801C05E
:10041000C79AEE246894E1F880B399270E2C02C0A5
:10042000959587950A94E2F780FD1FC0FF240E2D55
:10043000112788E230D180B39927002E02C095950C
:1004400087950A94E2F780FD04C0F394F4E0FF1569
:1004500080F785E0F81649F4E4E0EE1621F48F2DDC
:1004600029D1869902C08E2D86D0E394F5E0FE1541
:1004700098F6B299B1CF88EC0ED188EC0CD188EC0B
:100480000AD1B299A9CF8BE076D0A6CF80E887BBFE
:1004900082E081BB8FE788BB8DEF82BB41D108959D
:1004A000FF920F931F93CF93DF93CDB7DEB72197C2
:1004B0000FB6F894DEBF0FBECDBF082F192FFF2453
:1004C00059D1912F802F31D1198286E9E4D08C2F18
:1004D0009D2F019647D1082F192F6DE070E055D15F
:1004E000892BB9F06FE670E0912F802F5CD1892BBA
:1004F00019F080E090E013C062E770E0912F802F48
:1005000052D1892B19F081E090E009C083E090E09E
:1005100006C0F39489E08F15B8F682E090E021964A
:100520000FB6F894DEBF0FBECDBFDF91CF911F9104
:100530000F91FF9008951F93CF93C82F16E988233A
:100540000CF412E38C2F99278F779070892B71F020
:10055000C798812F84519FD0C79A812F9CD0C150BA
:100560008C2F99278F779070892B91F781E0A2D0FB
:10057000CF911F910895CF92DF92FF920F931F9317
:10058000CF93DF93CDB7DEB721970FB6F894DEBFD8
:100590000FBECDBFCC24DD24992784309105E9F02E
:1005A0008530910534F48230910549F0039771F05C
:1005B0002BC085309105C1F00B9701F125C00F2E9E
:1005C000F7E5CF2EF0E0DF2EF02D1EC00F2EF6EB5C
:1005D000CF2EF0E0DF2EF02D17C00F2EF5E1CF2E3D
:1005E000F1E0DF2EF02D10C00F2EF4E7CF2EF1E05A
:1005F000DF2EF02D09C082E09EDF22C00F2EF3ED2A
:10060000CF2EF1E0DF2EF02DC114D104B1F1B2D024
:1006100080E490E08AD01982FF2400E010E0FF20FF
:1006200079F48AE038D08C2F9D2F01969BD0082F2B
:10063000192FF39486E98F15F0F28981882389F3C5
:10064000F12FE02F80818E3349F081818E3331F09C
:1006500082818E3319F083E06EDF0FC08CE490E06E
:1006600064D080E690E070D09D2D8C2D5ED0C79830
:1006700086E920D086E91ED0C79A21960FB6F89455
:10068000DEBF0FBECDBFDF91CF911F910F91FF90C5
:10069000DF90CF900895982F882359F020E030E024
:1006A00086B32F5F3F4F82E020333807CCF3915061
:1006B000A9F70895CF93C82F882351F08AEFEBDF75
:1006C0008AEFE9DF8AEFE7DF8AEFE5DFC150B1F7B4
:1006D000CF9108951F920F920FB60F9211242F936E
:1006E0008F939F93EF93FF932091780089E790E099
:1006F000F92FE82FE20FF11D8CB18083822F8F5FDD
:1007000080937800803210F020937800FF91EF9171
:100710009F918F912F910F900FBE0F901F90189562
:1007200088E98AB98BE089B9089530E0F92FE82F7C
:10073000E30FF11DC895202D222329F02CB95D9BD4
:10074000FECF3F5FF3CF089520E0F92FE82FE20FAF
:10075000F11DE081EE2329F0ECB95D9BFECF2F5F08
:10076000F4CF0895F92FE82F80917800808389E7EE
:1007700090E00895F89480E2E9E7F0E011928A951C
:10078000E9F71092780078940895E82FF92F0190F6
:10079000061629F00020D9F7882799270895319760
:1007A0008E2F9F2F0895A82FB92FE62FF72F419155
:1007B000442309F40895E62FF72F41912D91222328
:1007C00071F024178A2F9B2FC9F74191442351F0D0
:1007D0002C91222321F0241771F71196F6CF882748
:0807E00099270895019708957F
:1007E8002B37383132313233343536370000004F49
:0807F8004B004552524F520024
:00000001FF
